:020000040000FA
:06000000D1EF03F0120035
:0600080004EF04F01200F9
:060018000CEF04F01200E1
:06002A000100CE070000FA
:080030006A000000020000005C
:08003800126A1E0E716E040134
:10004000400E096F200E0A6F040E0B6F880E086FAA
:100050000401200E0E6F040E0F6F400E0C6F120085
:10006000550EA76EAA0EA76EA68212000401140EEA
:10007000226F010E236F1200106A04012151105CDF
:100080001CE2166A176A22511024F36E23511620BF
:10009000F46E24511720F86EF4CFF7FFF3CFF6FF7C
:1000A0000800F550116E1050EA6A250FE96E040E33
:1000B000EA2211C0EFFF102AE0D7F86A1200F00E12
:1000C00004012217840EA66E106A04012151105CEF
:1000D00023E21050EA6A250FE96E040EEA22EFCF00
:1000E00018F01050156E166A176A22511024F36E1C
:1000F00023511620F46E24511720F86EF4CFF7FF29
:10010000F3CFF6FF18C0F5FF0C000F0E10140F0808
:1001100001E1A6DF102AD9D71200940EA66E106A4C
:1001200004012151105C1DE21050156E166A060E76
:10013000D89015361636E804FBE1176A16BE176824
:10014000040122511524F36E23511620F46E24511C
:100150001720F86EF4CFF7FFF3CFF6FF81DF102AF8
:10016000DFD7F86A1200A66A106A04012151105CF8
:100170000EE222511024A96EA6801050EA6A250FC3
:10018000E96E040EEA22A8CFEFFF102AEED7120084
:10019000106A04012151105C12E222511024A96E50
:1001A0001050EA6A250FE96E040EEA22EF50A86E9D
:1001B000040EA66E55DFA6B2FED7102AEAD71200AB
:1001C000C40EA66E106A04012151105C1FE210508B
:1001D000EA6A250FE96E040EEA22EFCF18F01050FC
:1001E000156E166A176A22511024F36E23511620D9
:1001F000F46E24511720F86EF4CFF7FFF3CFF6FF1B
:1002000018C0F5FF0C002CDF102ADDD7F86A1200A9
:1002100079D8060E015C03E36D50020B01E071D04A
:10022000120410E104010CBF0CD00401400E096F50
:10023000400E040108170401087D880E040108130C
:10024000126A5FD0040108BF5CD0106A040120511B
:10025000320A3BE0CD0A2DE0F80A27E0020A21E04D
:10026000010A1BE0070A15E0010A0FE0030A09E092
:10027000070A07E0060A01E035D0F8DE040E106E2A
:1002800032D0FADE050E10262ED019DF010E106EC8
:100290002AD043DF010E106E26D065DF050E102632
:1002A00022D076DF010E106E1ED08ADF010E106E96
:1002B0001AD06D96136A146A1306000E145A13505E
:1002C000141001E0F9D7FF000ED0030E0401215DE8
:1002D00002E1010E106E040E0401215D02E1010E27
:1002E000106E01D000D0010E126E10500AE010C046
:1002F0000DF4400E04010C1704010C7D880E04015E
:100300000C13120000016A516B1104E1200E6A6F98
:100310004E0E6B6F6A07000E6B5B6DA208D06A51C0
:100320006B112DE18B708B50010B12E125D0015028
:1003300002E18B9021D0010402E18B8009D0020EF2
:10034000015C02E18B8018D0030E015C03E18B900D
:100350008B821200050E015C05E16A516B110FE101
:100360008B700AD0060E015C0AE16A516B1107E13D
:100370008B708B50010B02E08B9212008B8212006B
:100380006C500BE1040100513C0BE842E8420D08BF
:1003900002E1D2EF01F0DAEF01F0040E6C5C01E152
:1003A00017D81200056A066A0B6A0C6AFBEC02F0A9
:1003B00058EF02F0020E055C09E157D8040100BDB8
:1003C00002D0C80E01D0880E006F120096EF02F026
:1003D000040E015C09E112C46EFF6E50000802E2D7
:1003E000050E01D0030E016E050409E10AD80401CF
:1003F00004BD02D0C80E01D0880E046F120096EF23
:1004000002F0080E0B5C000E0C5802E20B5001D0FB
:10041000080E0E6EE8CF05F4166AE8500B5E165013
:100420000C5A180E096E040E0A6E0E501DE002A240
:1004300007D007C0F6FF08C0F7FF0800F55005D049
:1004400007C0E9FF08C0EAFFEF50E66E09C0E9FF08
:100450000AC0EAFFE552E750EF6E072A000E0822B5
:10046000092A0A220E06E1D7120001C40FF00F502C
:100470000B240B6E000E0C200C6E180E076E040E73
:10048000086E0F5014E007C0E9FF08C0EAFFEF5004
:10049000E66E09C0E9FF0AC0EAFFE552E750EF6ED9
:1004A000092A000E0A22072A08220F06EAD712009C
:1004B0006D9806500BE10401080E016F100E026FDB
:1004C000040E036F840E006F04011ED0040110AFF0
:1004D0001DD00B50165D0C50175904E216C40BF0DA
:1004E00017C40CF08EDF010E056E0401080E016FBB
:1004F000100E026F040E036F800E006F0401180EC1
:10050000066F040E076FC80E046F1200020E056E10
:100510000401056BC80E046F0401080E016F180E6C
:10052000026F040E036FC80E006F1200056A04010B
:10053000080E016F100E026F040E036F8C0E006F19
:060540000401046B12002F
:0A054600080E6D6E6DBAFED7686AEC
:10055000110E696E020E016E12006850040B09E064
:100560006950040B06E06D92699468A402D0689407
:10057000FCD76850010B04E06950010B01E024D85E
:100580006850100B0AE06950100B07E06984689806
:100590006D82A19AA08A0300A19A6850200B06E000
:1005A0006950200B03E070B07090689A030E015CF4
:1005B00001E209D06850080B06E06950080B03E01F
:1005C000C0EC01F068961200686A7B0E696E6E6A74
:1005D000160E706E68A608D0689600000000000035
:1005E000000000000000F6D76D9896EC02F0036A58
:0605F000030E016E120073
:0A05F60004011051600BE842E842D6
:10060000E842E842E842000901E012001151080AFC
:100610002FE0010A2BE00F0A08E0030A01E01200B4
:10062000010E066E040E016E1200010E066E130519
:1006300006E13E0E076E070E086E120E11D0020E76
:10064000135D06E1500E076E070E086E200E08D0EF
:10065000030E135D08E1700E076E070E086E040EA0
:100660000B6E0C6A01D0066A0282120042EF03F0A0
:10067000010E066E030E076E000E086E0292010E4A
:100680000B6E1200010E066E12C403F0040112512B
:1006900003E1050E016E1200060E016E1CEF00F064
:1006A0002A0EF66E000EF76E000EF86E00010900BD
:1006B000F550656F0900F550666F03E1656701D07D
:1006C0003DD00900F550606F0900F550616F0900D9
:1006D000F550626F09000900F550E96E0900F55008
:1006E000EA6E090009000900F550636F0900F55032
:1006F000646F09000900F6CF67F0F7CF68F0F8CF14
:1007000069F060C0F6FF61C0F7FF62C0F8FF00014A
:10071000635302E1645307E00900F550EE6E63078E
:10072000F8E26407F9D767C0F6FF68C0F7FF69C051
:0E073000F8FF00016507000E665BBFD71200E0
:02073E001201A6
:10074000000200000008D8040B00010000000001B6
:1007500009022000010100803209040000020000AB
:10076000000007050102400000070581024000006B
:040770000403090471
:0C077400C150006E0F0EC11282A404D010
:100780000050C16E00EF04F08B6AFC0E946E140EE4
:100790006F6EA3EC02F0ADEC02F008EC01F0FBD7B9
:0207A000120045
:0E07A20013EE00F023EE00F0F86A1A9C50EC03
:0E07B00003F0E6EC03F0BAEC03F0FBD7120006
:0207BE0000EE4B
:0C07C00000F00F0EEE6AEA62FDD7120096
:0207CC00120019
:0207CE00000029
:06080000AEEF1BF0120038
:0608080035EF04F01200C0
:0608180022EF04F01200C3
:06082A00020094370000FB
:10083000B60200000200000037330000B8020000DA
:0408400001000000B3
:0C084400D8CFE4FFE0CFE4FFE46EDACF91
:10085000E4FFE2CFDAFFE652E552E5CFDAFFE550FA
:10086000E5CFE0FFE5CFD8FF1000DACFE4FFE2CF1D
:10087000DAFFE652E552E5CFDAFF1100D9CFE6FF05
:10088000E1CFD9FF020EE126C290070EB46E0F0E23
:10089000C16E8968926A8A68936A8B68946A8C6868
:1008A000956A8D6A010E966E0201010EAE6F02010D
:1008B000B669B7690201AC6B0201AD6B0201AA6BAC
:1008C0000201AB6BFA0ECB6ED08ECA949D829F92C2
:1008D000F28EF28C020EE15C02E2E16AE552E16E18
:1008E000E552E7CFD9FF1200D9CFE6FFE1CFD9FF1C
:1008F000020EE126010EDB6A0201806B0401040195
:100900001851800B6CE1060E0201B05D68E36D507A
:10091000020B65E10201806B040119510201805D47
:1009200053E202018051EA6A080FE96E050EEA22DD
:10093000EFCFDFFF0201B8511CE10D0E146EDF5046
:10094000145C05E00A0E156EDF50155C12E1020121
:10095000010EB86F0201AC51EA6A400FE96E020E57
:10096000EA220D0EEF6E0201AC2BDE52010EDD6E9F
:1009700015D00D0EDF5C11E00A0EDF5C0EE0020107
:10098000AC51EA6A400FE96E020EEA22DFCFEFFFB8
:100990000201B86B0201AC2B01D013D0400E020152
:1009A000AC5D02E10201AC6B0201AD510201AC5D34
:1009B00002E1228609D0010EDB5003E01CD9010EB2
:1009C000DB6A0201802BA8D70401400E196F400E8C
:1009D000040118170401187D880E04011813225011
:1009E00001E181D022A010D0770E146E310E156E69
:1009F000166A14C0E6FF15C0E6FF16C0E6FF47EC16
:100A00001AF0E552E552E55222A210D0710E146E92
:100A1000310E156E166A14C0E6FF15C0E6FF16C04B
:100A2000E6FF47EC1AF0E552E552E55222A410D059
:100A3000550E146E310E156E166A14C0E6FF15C001
:100A4000E6FF16C0E6FF47EC1AF0E552E552E55224
:100A500022A610D0390E146E310E156E166A14C00F
:100A6000E6FF15C0E6FF16C0E6FF47EC1AF0E552B8
:100A7000E552E55222A810D01A0E146E310E156EF2
:100A8000166A14C0E6FF15C0E6FF16C0E6FF47EC85
:100A90001AF0E552E552E55222AA00D022AC10D05D
:100AA000F90E146E300E156E166A14C0E6FF15C0EE
:100AB000E6FF16C0E6FF47EC1AF0E552E552E552B4
:100AC00022AE10D0E00E146E300E156E166A14C0F1
:100AD000E6FF15C0E6FF16C0E6FF47EC1AF0E55248
:100AE000E552E552226A35D8020EE15C02E2E16A83
:100AF000E552E16EE552E7CFD9FF1200D9CFE6FF0C
:100B0000E1CFD9FF0201AA51EA6A000FE96E020E95
:100B1000EA22FE0EDBCFEFFF0201AA2B400E0201FC
:100B2000AA5D02E10201AA6B0201AB510201AA5DBA
:100B300001E12284FE0EDBCF14F0156A14BE1568A5
:100B400014C0F3FF15C0F4FF00D0E552E7CFD9FF82
:100B50001200D9CFE6FFE1CFD9FFE6520201815161
:100B600045E1060E0201B05D41E36D50020B3EE12E
:100B70000201AA510201AB5D39E00201AB51020151
:100B8000D880AA551AE20201AB510201AA5DDF6EBC
:100B90000201AB510201826F836B000E02018227BA
:100BA000020E02018323DFCF86F20201876B02016E
:100BB000010E816FAAC2ABF219D0400E0201D8809B
:100BC000AB55DF6E0201AB510201826F836B000EE9
:100BD00002018227020E02018323DFCF86F2020187
:100BE000876B0201010E816F0201AB6BE552E5528A
:100BF000E7CFD9FF1200D9CFE6FFE1CFD9FF040E2E
:100C0000E126DE6ADD6A020EDB6A030EDB6A0201A0
:100C1000AD51EA6A400FE96E020EEA22EF50E66E2D
:100C2000E66A40EC1BF0E552E552020EF3CFDBFF23
:100C30000201AD2B400E0201AD5D02E10201AD6B80
:100C4000020EDB50DE6EDD6A0201AD51EA6A400F32
:100C5000E96E020EEA22EF502C0835E00201AD5198
:100C6000EA6A400FE96E020EEA22EF500D082BE00F
:100C70000201AD51EA6A400FE96E020EEA22EF501E
:100C8000E66EE66A40EC1BF0E552E552030EF3CF48
:100C9000DBFF0201AD2B400E0201AD5D02E102015E
:100CA000AD6B020EDBCF16F016C017F0166A030EFE
:100CB000DB5000011624146E000E1720156E14C0B0
:100CC000DEFF15C0DDFF000EDBCF08F0010EDBCF2D
:100CD00009F0500E081801E109501EE04F0E0818E7
:100CE00001E1095017E0550E081802E1430E0918FA
:100CF0000FE0520E081801E1095008E0560E0818DE
:100D000001E1095001E00AD009DA47D07DD845D089
:100D10007ED843D0BAD841D012DA3FD0030EDB5090
:100D20001AE1020EDBCFE6FFE66A020EDBCFE6FF3A
:100D3000E66ABD0E146E300E156E166A14C0E6FF1C
:100D400015C0E6FF16C0E6FF47EC1AF0176E070E57
:100D5000E15E175021D0030EDBCFE6FFE66A020EFC
:100D6000DBCFE6FFE66A030EDBCFE6FFE66A020EA4
:100D7000DBCFE6FFE66A950E146E300E156E166A2E
:100D800014C0E6FF15C0E6FF16C0E6FF47EC1AF0F8
:100D9000176E0B0EE15E175000D00201AD51EA6AEA
:100DA000400FE96E020EEA22EF500D080DE02250CE
:100DB0000BE1520E146E156ADF50141803E1DE5277
:100DC000DD50151801E0228EACC2ADF2040EE15CDC
:100DD00002E2E16AE552E16EE552E7CFD9FF120087
:100DE0000201AE5110E0140E146E370E156E166A25
:100DF00014C0E6FF15C0E6FF16C0E6FF47EC1AF088
:100E0000E552E552E552120039DDEADF1200D9CF92
:100E1000E6FFE1CFD9FF030EE126010EE66E07DB08
:100E2000E5520750DF6E020EE66E01DBE552DE5240
:100E300007C0DEFF08C0DDFFDD52225001E01BD0FD
:100E4000DF0418E1D950010FE96EDACFEAFFEE5066
:100E5000ED100BE0010E146E156A010EDB50141834
:100E600003E1020EDB50151804E1010EDBCFAEF2F8
:100E700001D0228CB5DF030EE15C02E2E16AE552AB
:100E8000E16EE552E7CFD9FF1200D9CFE6FFE1CFFF
:100E9000D9FF0E0EE126010EE66EC9DAE55207C053
:100EA00014F008C015F009C016F0070E141A050E4C
:100EB00014C0DBFF010EE66EBADAE55207C014F08B
:100EC00008C015F009C016F0070E141A060E14C05B
:100ED000DBFF010EE66EABDAE55207C014F008C086
:100EE00015F009C016F0070E141A070E14C0DBFF28
:100EF000010EE66E9CDAE55207C014F008C015F04A
:100F000009C016F0070E141A080E14C0DBFF010EFC
:100F1000E66E8DDAE55207C014F008C015F009C07E
:100F200016F0070E141A090E14C0DBFF010EE66E50
:100F30007EDAE55207C014F008C015F009C016F0BB
:100F4000070E141A0A0E14C0DBFF010EE66E6FDAEC
:100F5000E55207C014F008C015F009C016F0070EDE
:100F6000141A0B0E14C0DBFF010EE66E60DAE552B8
:100F700007C014F008C015F009C016F0070E141AC7
:100F80000C0E14C0DBFF010EE66E51DAE55207C00D
:100F900014F008C015F009C016F0030E141A0D0E57
:100FA00014C0DBFF225001E0AFD00D0EDB50030870
:100FB00002E3000E01D0010E146E0C0EDBCFE6FF33
:100FC0000B0EDBCFE6FF0A0EDBCFE6FF090EDBCF11
:100FD000E6FF080EDBCFE6FF070EDBCFE6FF060ECF
:100FE000DBCFE6FF050EDB50E552E710E552E710D8
:100FF000E552E710E552E710E552E710E552E71039
:10100000E552E710070802E3000E01D0010E1410AC
:1010100002E0228C79D0070EDB50010B100DF3CFCC
:1010200015F0060EDB50030B040DF3CF14F0050E84
:10103000DB50030B14101510DF6E0C0EDB50040B8D
:10104000100DF3CF19F00A0EDB50040B080DF3CF8F
:1010500018F0090EDB50040B040DF3CF17F0080E47
:10106000DB50040BE824166E070EDB50040B156EE4
:10107000060EDB50040BE8407F0B146E050EDB50B0
:10108000040BE840E8403F0B141015101610171021
:1010900018101910E76E010EE7CFDBFF0D0EDBCF46
:1010A000E6FF0A0EDB50030B400DF350E552E7104C
:1010B000E76E020EE7CFDBFF0C0EDB50030B400D9B
:1010C000F3CF16F00B0EDB50030B100DF3CF15F022
:1010D000090EDB50030B040DF3CF14F0080EDB50A8
:1010E000030B141015101610E76E030EE7CFDBFF8D
:1010F000DF50896E010EDB508A6E020EDB508B6E64
:10110000030EDB508C6E6CDE0E0EE15C02E2E16AD7
:10111000E552E16EE552E7CFD9FF12001C0E146EC6
:10112000370E156E166A14C0E6FF15C0E6FF16C02E
:10113000E6FF47EC1AF0E552E552E5521200D9CF2E
:10114000E6FFE1CFD9FF050EE126050EE66E6FD969
:10115000E5520750DF6E010EE66E69D9E552030EC7
:1011600007C0DBFF010EE66E62D9E552040E07C030
:10117000DBFF225001E051D1040EDB50020802E2F5
:10118000228C4BD1030EDB50050809E3030EDB5024
:1011900003080CE2470E146EDF50145C07E1030EE7
:1011A000DB50050802E2228C38D106D0030EDB505A
:1011B000030802E2228C31D1410E146EDF50145C20
:1011C0000AE1D950010FE96EDACFEAFF890EEE6E1F
:1011D0000F0EED6EC6D0420E146EDF50145C0AE1A5
:1011E000D950010FE96EDACFEAFF8A0EEE6E0F0ECC
:1011F000ED6EB7D0430E146EDF50145C14E1040E94
:10120000146E030EDBCFE7FF1450E726030EE7CF83
:10121000DBFFD950010FE96EDACFEAFF8A0EEE6EDE
:101220000F0EED6E9ED0440E146EDF50145C0AE17A
:10123000D950010FE96EDACFEAFF8C0EEE6E0F0E79
:10124000ED6E8FD0450E146EDF50145C14E1040E69
:10125000146E030EDBCFE7FF1450E726030EE7CF33
:10126000DBFFD950010FE96EDACFEAFF8C0EEE6E8C
:101270000F0EED6E76D0460E146EDF50145C30E12A
:10128000020EF36E030EDBCFF4FFF350F45C14E2B6
:10129000040E146E030EDBCFE7FF1450E726030E97
:1012A000E7CFDBFFD950010FE96EDACFEAFF890EF5
:1012B000EE6E0F0EED6E13D0020E146E030EDBCF2A
:1012C000E7FF1450E75E030EE7CFDBFFD950010FB5
:1012D000E96EDACFEAFF8D0EEE6E0F0EED6E41D0A5
:1012E000470E146EDF50145C3AE1030EDB500FE141
:1012F000020EF36E030EF3CFDBFFD950010FE96E40
:10130000DACFEAFF8D0EEE6E0F0EED6E27D0040ED3
:10131000F36E030EDBCFF4FFF350F45C0CE2030E2C
:10132000DB06D950010FE96EDACFEAFF8B0EEE6EC5
:101330000F0EED6E13D0020E146E030EDBCFE7FF1F
:101340001450E726030EE7CFDBFFD950010FE96EFB
:10135000DACFEAFF8B0EEE6E0F0EED6E02D0228C0E
:101360005CD0040EDB5015E1010EF36E030EDB5072
:1013700004E0D890F336E806FCE1F350E81C146E64
:10138000010EDBCFE9FF020EDBCFEAFF1450EF16B0
:1013900043D0040EDB0414E1010EF36E030EDB50A8
:1013A00004E0D890F336E806FCE1F350146E010E29
:1013B000DBCFE9FF020EDBCFEAFF1450EF122CD097
:1013C000010EF36E030EDB5004E0D890F336E8060E
:1013D000FCE1F350146E010EDBCFE9FF020EDBCF10
:1013E000EAFFEF501414E76E040EE7CFDBFF040EA4
:1013F000DBCFE6FFE66A8F0E146E300E156E166AAE
:1014000014C0E6FF15C0E6FF16C0E6FF47EC1AF071
:10141000176E050EE15E1750E3DC050EE15C02E29B
:10142000E16AE552E16EE552E7CFD9FF1200D9CF6C
:10143000E6FFE1CFD9FF040EE126030EDB6A0D0EB5
:10144000146E0201AD51EA6A400FE96E020EEA2203
:10145000EF50145C05E12288076A086A096A93D193
:101460000201AD51EA6A400FE96E020EEA22EF5026
:101470002C0820E00201AD51EA6A400FE96E020E2D
:10148000EA22EF50E66EE66A680E146E300E156EB4
:10149000166A14C0E6FF15C0E6FF16C0E6FF47EC6B
:1014A0001AF0176E050EE15E1750228A076A086A65
:1014B000096A69D10201AD2B400E0201AD5D02E166
:1014C0000201AD6B2D0E146E0201AD51EA6A400FA0
:1014D000E96E020EEA22EF50145C28E1040E156E4C
:1014E000FE0EDB50155C22E0050E166EFE0EDB5084
:1014F000165C1CE0FE0EDB0406E0030E146EFE0E0E
:10150000DB50145C06E1228C076A086A096A3BD149
:101510000DD0010EF36E030EF3CFDBFF0201AD2BF6
:10152000400E0201AD5D02E10201AD6B040E146ECE
:10153000FE0EDB50145C11E0050E156EFE0EDB5046
:10154000155C0BE0050EE66ED9CFE6FFDACFE6FFBD
:1015500024D9E552E552E5523AD00201AD51EA6A8A
:10156000400FE96E020EEA22EFCF14F0156A166AF8
:1015700014C0DFFF010E15C0DBFF020E16C0DBFF3B
:10158000050E146EFE0EDB50145C19E1000EDBCF6D
:10159000E6FF010EDBCFE6FF40EC1BF0E552E55223
:1015A000F3CF14F0F4CF15F0166A15BE166814C008
:1015B000DFFF010E15C0DBFF020E16C0DBFF0201CC
:1015C000AD2B400E0201AD5D02E10201AD6B030ED9
:1015D000DB5021E0DFCF14F0010EDBCF15F0020E5F
:1015E000DBCF16F00C680D680E6814C007F015C04C
:1015F00008F016C009F0BFEC18F004C014F005C0E4
:1016000015F006C016F014C0DFFF010E15C0DBFF99
:10161000020E16C0DBFFFE0EDB5026E1DFCF14F01A
:10162000010EDBCF15F0020EDBCF16F01634000EE4
:10163000161807E6D8807F0E1454000E1554000EBD
:10164000165401E28CD0D9CFE9FFDACFEAFF020EBF
:10165000D880EB50FF0A06E6800EEE5CFF0EEE58D7
:10166000FF0EEF5801E27BD0FE0EDB0424E1DFCF5A
:1016700017F0010EDBCF18F0020EDBCF19F0193492
:10168000000E191807E6D880FF0E1754000E1854E4
:10169000000E195464E3D9CFE9FFDACFEAFF020E56
:1016A000D890EB50000A06E6000EEE5C000EEE58F5
:1016B000000EEF5854E3020E1A6EFE0EDB501A5C59
:1016C00024E1DFCF1BF0010EDBCF1CF0020EDBCFDD
:1016D0001DF01D34000E1D1807E6D880FF0E1B54A8
:1016E0007F0E1C54000E1D543AE3D9CFE9FFDACF28
:1016F000EAFF020ED880EB50FF0A06E6000EEE5C11
:10170000800EEE58FF0EEF582AE3030E1E6EFE0EFB
:10171000DB501E5C29E1DFCF1FF0010EDBCF20F094
:10172000020EDBCF21F02134000E211807E6D8800D
:10173000FF0E1F54FF0E2054000E215410E3D9CF8A
:10174000E9FFDACFEAFF020ED890EB50000A06E676
:10175000000EEE5C000EEE58000EEF5805E2228CF3
:10176000076A086A096A0FD0DFCF14F0010EDBCFD9
:1017700015F0020EDBCF16F014C007F015C008F00C
:1017800016C009F000D0040EE15C02E2E16AE55205
:10179000E16EE552E7CFD9FF1200D9CFE6FFE1CFE6
:1017A000D9FF020EE126FD0EDBCFE9FFFE0EDBCFF7
:1017B000EAFFEE6AEE6AEE6A010EDB6AFC0EDB50AF
:1017C000F36E010EDBCFF4FFF350F45C55E202013F
:1017D000AD51EA6A400FE96E020EEA22EFCFDFFF59
:1017E000300EDF5C44E3DF50390841E3FD0EDBCF10
:1017F000E9FFFE0EDBCFEAFFEECF17F0EECF18F0D9
:10180000EFCF19F00A0E0C6E0D6A0E6A17C007F0C2
:1018100018C008F019C009F0BFEC18F004C017F0A8
:1018200005C018F006C019F0300EDF5C1A6E1B6A96
:101830001C6A17501A24146E18501B20156E19506C
:101840001C20166EFD0EDBCFE9FFFE0EDBCFEAFF9C
:1018500014C0EEFF15C0EEFF16C0EEFF0201AD2B67
:10186000400E0201AD5D02E10201AD6B02D0000E3F
:1018700005D0010EDB2AA2D7010E00D0146E020E95
:10188000E15C02E2E16AE552E16E1450E552E7CF15
:04189000D9FF12006A
:0C18940086EC11F0FB0EDBCFF3FFDB064F
:1018A000F35000090AE0D4EC11F0FA0E3FEC12F00C
:1018B000F3E1151CF1E1010E01D0000EB5EF11F0BE
:1018C00086EC11F03B0EE12402E3E168E652E16EA2
:1018D000010EDB6A020EDB6AF90EDBCFF6FFFA0EB1
:1018E000DBCFF7FFFB0EDBCFF8FF0800F550DF6E14
:1018F000DF5002E1D9EF10F0250EDF5C02E0CCEF03
:1019000010F0030EDB6A040EDB6A050EDB6A060EBE
:10191000DB6A070EDB6AEEEC10F02D0EDF5C0CE0EC
:101920002B0EDF5C09E0200EDF5C06E0230EDF5C9F
:1019300003E0300EDF5C1AE1DF50300A14E0130AD6
:101940000FE0030A0AE00B0A05E0060AE4E1030ED1
:10195000DB80E1D7030EDB82DED7030EDB84DBD72F
:10196000030EDB86D8D7030EDB88D5D72A0EDF5CC3
:101970001BE1EAEC10F038EC11F010E0030EDB8014
:1019800008680968130EDBCF0DF0140EDBCF0EF0E4
:1019900008EC19F0040E06C0DBFF03D0130E21EC97
:1019A00011F0EEEC10F00BD0090EDB6A8FEC11F0A9
:1019B00003E003EC12F0FAD7090E21EC11F0030E4C
:1019C000DBB0DB982E0EDF5C1BE1EEEC10F02A0E94
:1019D000DF5C0BE1EAEC10F038EC11F003E1130EE0
:1019E00073EC11F0EEEC10F00BD0090EDB6A8FEC0B
:1019F00011F003E003EC12F0FAD7090E73EC11F0CA
:101A0000680EDF5C07E1EEEC10F0680EDF5C1DE1B4
:101A1000030E18D0740EDF5C17E07A0EDF5C14E062
:101A2000480EDF5C06E0540EDF5C03E05A0EDF5C1C
:101A300002E1020E07D06C0EDF5C03E06A0EDF5C91
:101A400004E1010EC6EC11F0C9DBDF506E0A01E1C2
:101A50007FD31E0A01E192D1200A01E18FD13F0A12
:101A600001E149D11A0A01E146D10D0A01E143D150
:101A7000200A01E140D13A0A01E13DD1200A01E109
:101A80003AD1260A01E135D10D0A01E132D11A0A13
:101A900001E1D9D0200A4AE0300A1FE0460A0EE0F0
:101AA000250A01E083D3D950F90FE96EFF0EDA2041
:101AB000EA6E010EEE5E000EEE5AEE5AD4EC11F014
:101AC000250EE66E95DB03E1151C01E169D3D0EC30
:101AD00011F001E26BD3DB2A69D3080EDB6A040E36
:101AE000DB50010806E2040EDB0498EC11F0DB5039
:101AF0008BDB080EDB5009E0030EDB50010B05E128
:101B000072DB01E04DD3080EDB6A64DBEFCFDFFF51
:101B100048EC12F003E1151C01E142D3D0EC11F0C6
:101B200001E3DB2A60DB01E141D33AD3070EDB504E
:101B300002080FE114EC12F0030EDBEC11F00E0EB4
:101B4000EECFDBFF0F0EEECFDBFF100EEECFDBFF95
:101B500020D0F70EDBCF17F0F80EDBCF18F0020E17
:101B6000175E000E185AF70E17C0DBFFF80E18C0EC
:101B7000DBFF17C0E9FF18C0EAFFCBEC11F0166AD3
:101B80000E0E14C0DBFF0F0E15C0DBFF100E16C0CB
:101B9000DBFF0E0EDBCFE6FF0F0EDBCFE6FF100EF6
:101BA000DBCFE6FF1BEC1BF0E552E552E552130ECE
:101BB00007C0DBFF140E08C0DBFF060EDB5005E09C
:101BC000130E0FEC12F001E26ADB33EC12F002E2CA
:101BD000130E37DBF6EC11F006E0040E0FEC12F0FA
:101BE00002E2050E2EDB030EDBB005D0FCDA01E0CD
:101BF000D7D2080EDB6A090EDB6A0E0EDBCFF6FFCA
:101C00000F0EDBCFF7FF100EDBCFF8FF0800F5500B
:101C1000DF6EDF5014E039EC12F011E248EC12F004
:101C200003E1151C01E1BCD2BBDB01E3DB2A090E99
:101C3000DB2AD9500E0FE96E000ECBDBE7D7D3DAE3
:101C400001E1B4D2ADD2C6DA110EEECFDBFF120E37
:101C5000EDCFDBFF110EDBCFE6FF120EDBCFE6FF91
:101C60000DEC1BF0E552E552130EF3CFDBFF140E23
:101C7000F4CFDBFF060EDB5004E0130ED0DB01E2F5
:101C80000EDB33EC12F002E2130EDBDAAFDB05E021
:101C9000040EC5DB02E2050ED4DA030EDBB005D07C
:101CA000A2DA01E07DD2080EDB6A090EDB6A110EB2
:101CB000DBCFE9FF120EDBCFEAFFEFCFDFFFDF5014
:101CC00014E0D7DB12E2E4DB03E1151C01E168D28A
:101CD00067DB01E3DB2A090EDB2A110EDB2ADBCFEF
:101CE000E9FF120EE8E3DB2AE6D77DDA01E15ED2F6
:101CF00057D2030EDB8E070EDB0410E195DB040EDA
:101D00005ADB0A0EEECFDBFF0B0EEECFDBFF0C0E25
:101D1000EECFDBFF0D0EEECFDBFF6CD0070EDB50FE
:101D200003082CE1030EDBAE0DD0B2DA020E76DA38
:101D3000EFCF14F0156A166A176A14AE39D0156819
:101D4000166835D0F70EDBCF15F0F80EDBCF16F0A6
:101D5000020E155E000E165AF70E15C0DBFFF80EC8
:101D600016C0DBFF15C0E9FF16C0EAFFEFCF14F085
:101D70000A0E14C0DBFF0B0EDB6A38D0070EDB50F7
:101D8000020809E1030EDBAE04D059DB16AE10D019
:101D90000ED055DB0DD0030EDBAE12D079DA020E79
:101DA0003DDAF9DA166A176A15AE02D016681768B6
:101DB000E2DA0C0E16C0DBFF0D0E17C0DBFF1AD0E7
:101DC000F70EDBCF16F0F80EDBCF17F0020E165E23
:101DD000000E175AF70E16C0DBFFF80E17C0DBFF18
:101DE00016C0E9FF17C0EAFFD6DAC5DA0C0EDB6AC7
:101DF0000D0EDB6A060EDB5005E1010EF36E050EDB
:101E0000F3CFDBFF150EDB6A160EDB6AD950370FF6
:101E1000146E000EDA20156E390E14C0DBFF3A0E78
:101E200015C0DBFF380EDB6A080EDB6A0A0EAEDA7D
:101E3000DF50780A12E0200A10E0280A0CE0200A9D
:101E40000AE03F0A06E00D0A02E0200A08E1020E5D
:101E500005D0080E03D0080EDF26100E97DA030E09
:101E6000DBBE02D0DB92DB94DB50800B24E08ADA0D
:101E7000D890030EEB50000A08E6000EEE5C000E50
:101E8000EE58000EEE58000EEE5815E213DA0B680D
:101E90000C680D680E68D5EC1AF00A0E02C0DBFF64
:101EA0000B0E03C0DBFF0C0E04C0DBFF0D0E05C0E4
:101EB000DBFF2D0E08D0030EDBA202D02B0E03D0C9
:101EC000DBA408D0200EF36E170EF3CFDBFF150E48
:101ED000DB2A02D0170EDB6A050EDB5003E1B7D90F
:101EE00001E189D0740E146E370E156E000E166E59
:101EF000070EDBCF17F0186A196A1A6A17C00BF0C1
:101F000018C00CF019C00DF01AC00EF0D3D966EC51
:101F10001BF014500224F36E15500320F46E16507B
:101F20000420F86EF4CFF7FFF3CFF6FF0800090E98
:101F3000F5CFDBFF580EDF5C0FE1610EF36E090E8B
:101F40007BD90AE3200E146E090EDBCFE7FF145095
:101F5000E75E090EE7CFDBFF070EDBCF14F0156A53
:101F6000166A176A0FDA14C00BF015C00CF016C011
:101F70000DF017C00EF0EECF06F0EECF07F0EECF6B
:101F800008F0EFCF09F066EC1BF009C0EDFF08C0C8
:101F9000EDFF07C0EDFF06C0EFFF390EDBCFE9FF15
:101FA000DB063A0EDBCFEAFF01E2DB06090EDBCFF0
:101FB000EFFF150EDB2A4BD995E1030EDBA61DD0F2
:101FC0006F0EDF5C06E1C1D918E3150EDB285BDA82
:101FD00014D0780EDF5C09E0580EDF5C06E0620E7C
:101FE000DF5C03E0420EDF5C08E1020EF36E160ECA
:101FF000F3CFDBFF02D0150EDB6A030EDB50100BB4
:102000000EE0040EDBCF14F0050EDB50D880145424
:1020100006E2060EDB5003E1040EDB5034DA95D9FC
:102020000AE2050EDBCFE7FF150EDB50E75E050E7B
:10203000E7CFDBFF02D0050EDB6A040EDBCF14F026
:10204000160E45D9D880145414E2160EDBCFE6FFE5
:10205000150EDBCFE6FF040EDBCFE6FF050EDB50EF
:10206000E552E75CE552D880E754E552D880E75462
:102070005FD9030EDB50010B0BE1080EDB5008E0CB
:10208000B2D801E08DD0080EDB50BED8080EDB6A56
:10209000170EDB5007E088D9170EF1D903E1151CA4
:1020A00001E17ED0160EDB5016E07ED9300EE66ED2
:1020B0009FD802E1151C74E077D9DFCFE6FF93ECDF
:1020C0001AF0E552E552E552F4CF15F00001F31C89
:1020D00002E1151C65E0050EDBCF14F0160EDB5097
:1020E000D880145409E2050EDBCFE7FF160EDB5053
:1020F000E75E050EE7CFDBFF300EE66E050ECBD9AF
:102100004FE1390EDB2ADBCFE9FF3A0E01E3DB2A90
:10211000DBCFEAFF090EEFCFDBFFDB500EE044D947
:10212000090EADD902E1151C3BE0390EDB2ADBCFED
:10213000E9FF3A0EEDE3DB2AEBD755D831E1160E75
:10214000DBCFE6FF080EC3D8E552E7245DD82ED0DA
:10215000070EDB50030A1CE0010A14E0030A07E043
:102160007BD9DBCFEEFF020EDBCFEDFF1FD0F5D822
:10217000196A17AE02D0186819682CD8BCD819C0D3
:10218000EEFF14D0EAD817BE186824D8B4D80ED001
:1021900063D9DBCFEFFF0AD07BD905E1151C03E142
:1021A000F368F46810D0FCD801E3DB2A79D975EF25
:1021B0000CF0010EDBCF14F0020EDBCF15F014C0D3
:1021C000F3FF15C0F4FF3B0EE15C02E2E16AE55269
:1021D000E16ECBD029D9020EDBEF11F061D90800F6
:1021E000F550DF6E1200200EE66E080E4BEF12F077
:1021F00093EC1AF0E552E552E552F3CF14F0F4CF28
:1022000015F00001F31C1200146E156AD950010F6D
:102210004DD91450EE261550ED221200185E000E16
:10222000195AF70E18C0DBFFF80E19C0DBFF18C0F3
:10223000E9FF19C0EAFF1200DBCFF4FFF350F45CB2
:102240001200DB50E76E040EE7CFDBFF12000A0E30
:10225000DBCF14F00B0EDBCF15F00C0EDBCF16F03E
:102260000D0EDBCF17F014501510161017101200BA
:10227000130EEECFDBFF140EEDCFDBFF130EDBCF23
:1022800014F0140EDBCF15F00001800E15141200AF
:10229000F70EDBCF18F0F80EDBCF19F01200050EA9
:1022A000DB50E66ED950130F01D9E552E750EE6EC0
:1022B000ED6A12000A0EDBCF06F00B0EDBCF07F043
:1022C0000C0EDBCF08F00D0EDBCF09F01200DBCFD8
:1022D000E6FF150EDBCFE6FF050EDB50E552E724E7
:1022E000E552E7241200DB50CED8010EF36E060E45
:1022F000F3CFDBFF1200EE50EFCFEAFFE96E16C01E
:10230000EEFF17C0EEFF18C0EEFF1200D9CFE6FFB8
:10231000DACFE6FFE1CFD9FFE2CFDAFF1200DFCF5D
:10232000E6FFE66A54EC1BF0E552E552F35012006A
:10233000E76E080EE7CFDBFF1200EECF14F0EECF12
:1023400015F0EFCF16F0176A1200050EDBCF14F070
:10235000150EDB50D88014541200010EDBCF16F09E
:10236000020EDBCF17F0186A1200E552E5CFDAFF54
:10237000E7CFD9FF12000A0E14C0DBFF0B0E15C009
:10238000DBFF1200D9500A0F56EF12F0F36E070E62
:10239000F3CFDBFF1200EECF14F0EFCF15F01200F9
:1023A000010EDB2A020E1200FC0EDBCFE6FFFD0E53
:1023B000DBCFE6FF1200145E000E155AF70E14C0B4
:1023C000DBFFF80E15C0DBFF14C0E9FF15C0EAFF04
:1023D0001200DA20EA6EEF2AEECFF6FF000EEF22AF
:1023E000EECFF7FFEF22EECFF8FF1200040EDBCFA7
:1023F000E6FF130EDB50E552E75C9ADFDB5004DFAB
:10240000060EDB501200090EDB500A0DF350DF24DC
:10241000D00FE76E090EE7CFDBFFEEEF10F0DB50D9
:10242000F36E050E1CEF11F0F70EDBCF14F0F80E73
:10243000DBCF15F01200DFCFE6FFF8EF10F028DF5A
:10244000030EECDE9DEF11F04AEC0CF0E552E55284
:10245000E552E55200091200BDDEEE50EFCFEAFF73
:10246000E96E010E1200130EDB50F36E040E1CEF2A
:1024700011F0040EDB50F36E090E1CEF11F0DBCFF0
:10248000E6FFF8EF10F0E76E050EE7CFDBFF120076
:102490008BDF1BEF12F0DBCFE6FF86DF24EF12F0BD
:1024A000D950F90FE96EFF0EE9EF11F0E96E000E59
:0624B000DA20EA6E1200C2
:0A24B600040120511F0B010801E092
:1024C00060D004012051600BE842E842E842E84253
:1024D000E842010801E055D00401245104E0040160
:1024E000240501E04ED004012151230A48E0010AED
:1024F00040E0030A30E0010A25E0240A22E0070A4E
:102500001FE0010A1CE0030A11E0010A01E038D0D3
:102510000201030EA36F0201900EA46F020EA56FBD
:102520000201B1930201080EA86F2BD00201030E25
:10253000A36F0201900EA66F020EA76F22D021D0CA
:1025400020D01FD00201030EA36F0201880EA66FD8
:10255000020EA76F16D00201030EA36F0201880EB0
:10256000A46F020EA56F0201B1930201070EA86FBE
:1025700008D00201030EA36F22C48FF202D001D053
:1025800000D012000201886BC20E896F010E8A6FA3
:102590008B6B02018C6B02018D6B0201080E8E6F3A
:1025A0000201816B0201806B1A0E726E1E0E736E39
:1025B0000401000E166F050E176F0401400E146F14
:1025C0000401400E196F0401080E1A6F050E1B6FEF
:1025D0000401880E186F0401480E1E6F050E1F6F50
:1025E0000401400E1C6F1200D9CFE6FFE1CFD9FFE6
:1025F0000201806B040118BF39D0FC0EDBCF14F050
:1026000004011951D880145403E2FC0E19C4DBFFF5
:102610000201806BFC0EDB500201805D1CE20201B6
:102620008051EA6A080FE96E050EEA22EF50E66E65
:1026300002018051E76EFD0EDBCFE9FFFE0EDBCF1E
:10264000EAFFE750E926000EEA22E552E750EF6E76
:102650000201802BDFD70401400E196F400E0401E8
:1026600018170401187D880E040118130201805107
:1026700000D0E552E7CFD9FF1200D9CFE6FFE1CF76
:10268000D9FFE6520201815101E031D0DF6ADF2A31
:10269000DF50146E156A145002E1010E151801E1A5
:1026A0000BD0FD0EDBCFE9FFDB2AFE0EDBCFEAFF0E
:1026B00001E3DB2AEF50EBE1DF50146E156AD950CD
:1026C000FD0FE96EFF0EDA20EA6E1450EE5E155033
:1026D000ED5ADF06FD0EDBCF82F2FE0EDBCF83F27A
:1026E000DFCF86F20201876B0201010E816FE55296
:1026F000E552E7CFD9FF1200D9CFE6FFE1CFD9FFEE
:10270000E6520201815101E033D0DF6ADF2ADF5057
:10271000146E156AFF0E141801E1155001E10CD07A
:10272000FD0EDBCFF6FFDB2AFE0EDBCFF7FF01E36A
:10273000DB2A0800F550EAE1DF50146E156AD95023
:10274000FD0FE96EFF0EDA20EA6E1450EE5E1550B2
:10275000ED5ADF06FD0EDBCF82F2FE0EDBCF83F2F9
:10276000DFCF86F20201010E876F0201010E816F39
:10277000E552E552E7CFD9FF1200D9CFE6FFE1CF0E
:10278000D9FFE65204011CBF7DD0030E0201815D1A
:1027900002E10201816B0201815101E173D0020E5D
:1027A0000201815D06E104011D6B0201030E816FD0
:1027B00061D0020181055EE1400E146E156A0201CE
:1027C0008651145C000E155803E2400EDF6E02D0F5
:1027D00086C2DFFFDFCF1DF4DF500201865D0201FC
:1027E000866F0201480E846F050E856F0201870512
:1027F00018E1DF5015E082C2F6FF83C2F7FF080040
:10280000F55084C2E9FF85C2EAFFEF6E0201842B16
:10281000000E85230201822B000E8323DF06E9D7F9
:1028200016D0DF5014E082C2E9FF83C2EAFFEF5006
:1028300084C2E9FF85C2EAFFEF6E0201842B000E1D
:1028400085230201822B000E8323DF06EAD70201D3
:10285000865110E104011D51146E156A400E1418C2
:1028600001E1155004E10201020E816F03D0020163
:10287000030E816F400E04011C1704011C7D880E9D
:0E28800004011C13E552E552E7CFD9FF120008
:02288E006C508C
:1028900002E0000E01D0010E00090BE0040100511E
:1028A0003C0BE842E8420D0802E10CD801D042D8C6
:1028B00008D06C5002E0000E01D0010E040901E0C6
:1028C0004BD81200D9CFE6FFE1CFD9FFE652020183
:1028D000A26B0201A36B0201A86BA96BE4EC15F0DB
:1028E000DF6ADF50146E156A010E145C000E155875
:1028F0001BE20201A35101E017D0F76ADF34FE0B9F
:10290000F736F66E350EF626330EF7220900F5CFB0
:1029100014F00800F5CF15F004D015C0FAFF1450DC
:10292000F96EFBDFDF2ADDD7F0D8E552E552E7CFBD
:10293000D9FF1200020E0201A25D0CE1A4D804012D
:1029400000BD04D00401C80E006F03D00401880E3E
:10295000006F01D029D91200040E0201B05D0CE114
:1029600022C46EFF6E50000804E20201050EB06F33
:1029700003D00201030EB06F0201A2050CE10DD8D5
:10298000040104BD04D00401C80E046F03D0040187
:10299000880E046F01D008D91200D9CFE6FFE1CF2D
:1029A000D9FF020EE1260201080EA85D000EA9590A
:1029B00005E2A8C2DEFFA9C2DDFF03D0080EDE6E6D
:1029C000DD6A0401049304010491010EDB5004014B
:1029D0000413DFCF05F4000EDB500201A85F010EE7
:1029E000DB500201A95B0201280EA66F040EA76F3F
:1029F0000201B1A320D0D9CFE9FFDACFEAFFEE5030
:102A0000ED1018E0A4C2F6FFA5C2F7FF0800F550CC
:102A1000A6C2E9FFA7C2EAFFEF6E0201A62B000ED5
:102A2000A7230201A42B000EA523DF06010E01E25D
:102A3000DB06E1D71ED0D9CFE9FFDACFEAFFEE50AF
:102A4000ED1017E0A4C2E9FFA5C2EAFFEF50A6C24D
:102A5000E9FFA7C2EAFFEF6E0201A62B000EA72333
:102A60000201A42B000EA523DF06010E01E2DB0606
:102A7000E2D7020EE15C02E2E16AE552E16EE55264
:102A8000E7CFD9FF1200D9CFE6FFE1CFD9FF020E81
:102A9000E126030E04010015E76E010EE7CFDBFF10
:102AA00001C4DFFFDE500201A827DD500201A92387
:102AB0000201280EA46F040EA56FD9CFE9FFDACF6B
:102AC000EAFFEE50ED1017E0A4C2E9FFA5C2EAFF4D
:102AD000EF50A6C2E9FFA7C2EAFFEF6E0201A62BE4
:102AE000000EA7230201A42B000EA523DF06010E72
:102AF00001E2DB06E2D7020EE15C02E2E16AE552A6
:102B0000E16EE552E7CFD9FF12006D980201A351A3
:102B10000FE10401080E016F0401200E026F040E84
:102B2000036F0401840E006F0401840E046F3BD018
:102B3000040120AF25D00201A8510401265D020145
:102B4000A9510401275904E226C4A8F227C4A9F216
:102B500024DF0201010EA26F0401080E016F0401BF
:102B6000200E026F040E036F0401800E006F04013B
:102B7000280E066F040E076F0401C80E046F13D0F1
:102B80000201020EA26F0401056B0401C80E046F5E
:102B90000401080E016F0401280E026F040E036F7A
:102BA0000401C80E006F12000201A26B0401080E9E
:102BB000016F0401200E026F040E036F0401880EE2
:082BC000006F0401046B120018
:082BC80004012051600BE842FA
:102BD000E842E842E842E842000901E058D0040136
:102BE0002151070A53E00B0A51E0070A42E0010AAB
:102BF0002CE00B0A28E0020A26E0030A22E0080A79
:102C000012E0010A0EE00F0A0AE0030A01E03ED0DA
:102C10000201010EA36F0201040EB06F38D038D844
:102C200036D093D834D00201010EA36F0201B20E48
:102C3000A46F020EA56F0201B1930201010EA86FED
:102C400026D0ABD824D0F9D822D00201010EA36F30
:102C5000040124510201A46FA56BB30E0201A42745
:102C6000020E0201A5230201B1930201010EA86F19
:102C70000ED00201010EA36F04012451EA6AB30FC2
:102C8000E96E020EEA2222C4EFFF01D000D012004A
:102C9000800E0401205D58E104012351030A34E051
:102CA000010A10E0030A01E04DD00201010EA36FFA
:102CB00002016A0EA46F320EA56F120E0201A86FF8
:102CC000A96B40D00201010EA36F04012251F66EE0
:102CD000F76AD890F636F7362B0EF626330EF72223
:102CE0000900F5CFA4F20A00F5CFA5F2020E020109
:102CF000F76AA425F66EA551F7220900F5CFA8F2D0
:102D00000A00F5CFA9F21ED00201010EA36F040143
:102D10002251F66EF76AD890F636F7362F0EF62661
:102D2000330EF7220900F5CFA4F20A00F5CFA5F281
:102D3000A4C2F6FFA5C2F7FF0800F5500201A86F74
:102D4000A96B00D00201B18312000201010EA36F32
:102D50000F0EE66E710EE66E0F0EE66E1FEC18F0AB
:102D6000E552E552E552010EE66EB30EE66E020E36
:102D7000E66E1FEC18F0E552E552E55222C4B2F2BD
:102D80000401225104E10201050EB06F05D00201D9
:102D9000060EB06FC2EC12F012000401286B0401A1
:102DA000296B040120511F0B020A14E0030A0EE0F4
:102DB000010A01E034D00201010EA36F0401288151
:102DC0000201B1A102D00401288329D00201010E21
:102DD000A36F25D00201010EA36F040124510F0B34
:102DE000080DF350156A000F146E040E152204012D
:102DF0002451800B01E0010E040DF3500201142454
:102E0000A66F000E1520A76FA6C2E9FFA7C2EAFFB2
:102E1000EF50040B03E00401010E286F00D0020103
:102E2000A3050AE10201280EA46F040EA56F02019A
:102E3000B1930201020EA86F12000401220511E1F4
:102E4000040120511F0B00090CE10201010EA36FC8
:102E5000030E0401215D03E10201B18102D00201F0
:102E6000B191040122513EE1040120511F0B0208DF
:102E700039E1040124510F0B000934E00201010E75
:102E8000A36F040124510F0B080DF350156A000FB6
:102E9000146E040E152204012451800B01E0010E72
:102EA000040DF35002011424A66F000E1520A76F25
:102EB000030E0401215D07E1840EA6C2E9FFA7C24B
:102EC000EAFFEF6E0FD0040124AF06D0A6C2E9FFDF
:102ED000A7C2EAFFEF6A06D0880EA6C2E9FFA7C222
:062EE000EAFFEF6E120094
:0A2EE6006DA610D802D06DB614D806
:102EF0000201B00509E16DBA07D0686A696A6980A4
:102F000069880201020EB06F12006D6A696A6D86EF
:102F10000201010EB06F12006D6A696A0201B06BA6
:102F20001200FADF12000201B05101E13AD06850FC
:102F3000040B04E06950040B01E03CD86DB231D0C1
:102F40006850010B04E06950010B01E056D868504D
:102F5000100B04E06950100B01E024D86850400BBE
:102F600004E06950400B01E03DD86850200B04E0BC
:102F70006950200B01E038D86850020B04E069501A
:102F8000020B01E038D8030E0201B05D01E209D066
:102F90006850080B06E06950080B03E047EC14F09A
:102FA00068961200698468986D82A19AA08A0300CD
:102FB000A09A12006D926994689412000201B1A166
:102FC00010D0F8DF6D840201080EB46F070EB56FE4
:102FD0000201B407000EB55B0201B451B511F8E16E
:102FE0006D941200689C120070A003D0D4EC15F010
:102FF0007090689A1200689212006A6A686A9F0E5E
:103000006B6E7B0E696E6E6A0F0EE66E710EE66E6B
:103010000F0EE66E14D8E552E552E552160E706EAC
:1030200068A602D06896FCD76D98D4EC15F0020122
:10303000B1910201B26B0201030EB06F1200D9CF41
:10304000E6FFE1CFD9FFFD0EDBCFE9FFFE0EDBCFC0
:10305000EAFFFC0EDB5004E0EE6AFC0EDB06F9D75B
:08306000E552E7CFD9FF120091
:083068002135204572723A2067
:103070004E65656420636F6D6D61206E6578742C9C
:1030800020666F756E643A20272563270D0A002598
:1030900031750D0A002138204572723A20556E6B49
:1030A0006E6F776E20636F6D6D616E642027256390
:1030B00025633A253258253258270D0A0021382039
:1030C0004572723A20556E6B6E6F776E20636F6D2E
:1030D0006D616E64202725633A253258270D0A005A
:1030E0002137204572723A204578747261207061F0
:1030F000726D617465720D0A002136204572723A54
:1031000020496E76616C696420706172616D7465CE
:10311000722076616C75650D0A002134204572724B
:103120003A204D697373696E6720706172616D65D5
:103130007465722873290D0A002133204572723A92
:1031400020525820427566666572206F76657272ED
:10315000756E0D0A002132204572723A20545820B3
:10316000427566666572206F76657272756E0D0ABD
:0D317000002131200D0A002130200D0A0041
:02317E0009C086
:1031800013F008C012F007C011F007500C02F4CF82
:1031900005F0F3CF04F008500D02F4CF07F0F3CFA1
:1031A00006F00C02F3500526F4500622E86A0722C6
:1031B00011500D02F3500526F4500622E86A07224A
:1031C00009500C02F3500626F450072209500D0254
:1031D000086AE86A0822F3500726F45008221150C2
:1031E0000E02F3500626F4500722096AE86A082204
:1031F000092212500E02F3500726F4500822E86A02
:10320000092213500E02F3500826F4500922000C34
:1032100009C013F008C012F008500D02F4CF07F0F7
:10322000F3CF06F009500E02F4CF09F0F3CF08F007
:103230000D02F3500726F4500822E86A09221250C2
:103240000E02F3500726F4500822E86A09220EAE57
:103250002EEF19F01250085E1350095A13AE000CED
:0A3260000D50085E0E50095A000CD4
:06326A0012010002020047
:103270000008D8040A00000001020001090243000E
:10328000020100803209040000010202010005244D
:103290000010010424020205240600010524010097
:1032A000010705820308000209040100020A000068
:1032B00000070503024000000705830240000004E8
:1032C00003090434034D006900630072006F00635A
:1032D0000068006900700020005400650063006809
:1032E000006E006F006C006F0067007900200049DD
:1032F000006E0063002E00340343004400430020AE
:1033000000520053002D00320033003200200045EF
:10331000006D0075006C006100740069006F006E44
:10332000002000440065006D006F007C327C32BFDD
:0733300032C332F732B6246C
:013337000095
:083338000F0EC16E010E966E2E
:1033400084A03AD08D6A926A89689368946AC30EA1
:103350008B6E956A8C68040E8114040DF3CF15F002
:10336000020E8114E824146E010E8114141015103D
:10337000FF0A896E200E8114E824FF0A8B6E800EEE
:103380008114E8407F0B166E400E8114E840E8403F
:103390003F0B156E100E8114E840E8403F0B146E91
:1033A000080E8114E840E840E8401F0B1410151087
:1033B0001610FF0A8C6ECFD705D811D874EC04F024
:1033C000FCD712000F0EC112140E6F6E0201B06B0B
:1033D0000201B16B0201B26B3EEC04F0120073EC1F
:1033E00017F06FBE02D093EC17F0BDEC13F0120093
:1033F0002A0EF66E080EF76E000EF86E0201090036
:10340000F5509D6F0900F5509E6F03E19D6701D057
:103410003DD00900F550986F0900F550996F0900EB
:10342000F5509A6F09000900F550E96E0900F55052
:10343000EA6E090009000900F5509B6F0900F5507C
:103440009C6F09000900F6CF9FF2F7CFA0F2F8CFEA
:10345000A1F298C2F6FF99C2F7FF9AC2F8FF0201E3
:103460009B5302E19C5307E00900F550EE6E9B0769
:10347000F8E29C07F9D79FC2F6FFA0C2F7FFA1C2EE
:0E348000F8FF02019D07000E9E5BBFD71200F1
:02348E00D9CF94
:10349000E6FFDACFE6FFE1CFD9FFE2CFDAFFE6526F
:1034A000E652E652E652D950FB0F146EFF0EDA20B8
:1034B000156E14C0DEFFDD6EDECFE6FFDDCFE6FF6A
:1034C000FB0EDBCFE6FFFC0EDBCFE6FFFD0EDBCF16
:1034D000E6FFB6C2E6FFB7C2E6FF60EC0CF0146E82
:1034E000070EE15C02E2E16AE552E16E1450020E61
:1034F000F3CFDBFF030EF4CFDBFF020EDBCF14F0C4
:10350000030EDBCF15F014C0F3FF15C0F4FF040E5B
:10351000E15C02E2E16AE552E16EE552E5CFDAFFF5
:06352000E7CFD9FF120005
:0A352600D9CFE6FFDACFE6FFE1CFD0
:10353000D9FFE2CFDAFFFB0EDBCF14F0FC0EDBCFBE
:1035400015F00001800E15141AE1FB0EDBCFE9FF28
:10355000FC0EDBCFEAFFEECFF3FFEDCFF4FFEE2A58
:10356000000EEF22F3CFE9FFF4CFEAFFFD0EDBCF31
:10357000EFFFEF50156AF36E15C0F4FF10D0FB0E8D
:10358000DB50FE0806E1FD0EDBCFE6FFA0EC1BF0F2
:1035900005D0FD0EDBCFE6FF7EEC05F0E552E552EF
:0A35A000E5CFDAFFE7CFD9FF1200F4
:0635AA0006500B02F3CFF6
:1035B00002F0F4CF03F00C02F3500326000EF420C7
:1035C000046E06500D02F3500426000EF420056E22
:1035D00006500E02F350052607500B02F350032647
:1035E000F4500422000E052207500C02F35004266A
:1035F000F450052207500D02F350052608500B0227
:10360000F3500426F450052208500C02F35005260E
:0A36100009500B02F35005261200CA
:06361A00FE0EE3CFE9FF04
:10362000FF0EE3CFEAFFF36AF46AEE5203E0F34AD7
:10363000F42AFBD71200FF0EE3CFF8FFE552FF0E8E
:10364000E3CFF7FFE552FF0EE3CFF6FFE552E66A60
:10365000E66AE66A0900F55209E0FD0EE32A05E193
:10366000FE0EE32A02E1FF0EE32AF4D7FD0EE3CFBC
:1036700007F0FE0EE3CF08F0FF0EE3CF09F01200D3
:10368000FF0EE124E96EFF0EE220EA6EEDCFF4FFBB
:10369000EFCFF3FFF46607D0600EF36404D07B0E27
:1036A000F36001D0F39A1200F36AF46AFF0EE1248A
:1036B000E96EFF0EE220EA6EED6607D02F0EEF6492
:0C36C00004D03A0EEF6001D0F32A120093
:0436CC00056A046A1D
:1036D000036A026A200EE76ED8900636073608366F
:1036E000093602360336043605360B50025C0C50A0
:1036F00003580D5004580E50055809E30B50025E54
:103700000C50035A0D50045A0E50055A062AE72E43
:04371000E4D71200E8
:0C3714004F4B0D0A000D0A00446967418C
:103720007274732054616C6C7920436F6E74726F85
:0F3730006C6C65722058442076302E350D0A00DF
:10374000FF0EE350ACBA04D0AF6AAB8EAC8A949C47
:0C375000ACA2FED7AD6EF36EF46A12005E
:04375C0013EE00F078
:1037600023EE00F0F86A019CF8EC19F09CEC19F0DB
:04377000FDD712006F
:0C37740030313233343536373839616279
:053780006364656600B2
:0A37860000EE00F00F0EEE6AEA629A
:04379000FDD712004F
:02379400FEFF36
:020000040030CA
:0100000024DB
:010001000EF0
:010002003AC3
:010003001EDE
:010005008179
:010006008178
:010008000FE8
:010009008076
:01000A000FE6
:01000B00A054
:01000C000FE4
:01000D0040B2
:00000001FF
